:040000006F30101D30
:10000400000000000000000022370000423700001A
:1000140000000000CE3900000000000000000000D5
:10002400CE390000CE3900000000000000000000BE
:100034000C2F0000000000009002000000000000EF
:10004400CE390000CE390000CE390000CE39000090
:10005400CE390000CE390000023300002A330000FC
:10006400523300007A330000A2330000CE3900007E
:10007400CE390000CE390000CE390000CE39000060
:10008400CE390000CE390000CE390000CE39000050
:10009400CE390000CE390000CE390000CA3300004A
:1000A400CE390000CE390000CE390000CE39000030
:1000B400CE390000CE390000CE390000CE39000020
:1000C400CE390000CE390000CE390000CE39000010
:1000D400CE390000DA360000CE390000CE390000F7
:1000E4003C340000CE390000CE390000CE39000087
:1000F400CE390000CE390000CE390000CE390000E0
:1001040000000000CE390000CE390000CE390000D6
:10011400CE390000CE390000CE390000CE390000BF
:10012400CE390000CE390000CE390000CE390000AF
:10013400CE390000CE390000CE390000CE3900009F
:10014400CE390000CE390000CE390000CE3900008F
:10015400CE390000CE390000CE390000CE3900007F
:10016400CE390000CE390000CE390000CE3900006F
:10017400CE390000CE390000CE390000CE3900005F
:10018400CE390000CE390000CE390000CE3900004F
:10019400CE390000CE390000CE390000CE3900003F
:1001A400000000000000000000000000000000004B
:0C01B4000000000000000000000000003F
:1001C00097020120938202E4938202E0739002344A
:1001D00003210500224573100530B1A819712320B1
:1001E000250006C006C216CAF322003093F2820030
:1001F000638402009302000816C412C81ACC1ECEF3
:1002000022D026D22AD42ED632D836DA3ADC3EDEB6
:10021000C2C0C6C2CAC4CEC6D2C8D6CADACCDECE26
:10022000E2D0E6D2EAD4EED6F2D8F6DAFADCFEDE96
:1002300003A1050009A002457310153492403785CB
:10024000000013050580732005302245732005301A
:100250004242D2426243F243025492542255B25572
:100260004256D2566257F257064896482649B64932
:10027000464AD64A664BF64B065C965C265DB65DF2
:10028000465ED65E665FF65F09617300203000004F
:10029000197116CA9302000816C49302000273A0D3
:1002A000428006C212C81ACC1ECE22D026D22AD430
:1002B0002ED632D836DA3ADC3EDEC2C0C6C2CAC456
:1002C000CEC6D2C8D6CADACCDECEE2D0E6D2EAD4E6
:1002D000EED6F2D8F6DAFADCFEDE73110134FD2335
:1002E000EF107001EF0040617311013413848189B4
:1002F0000329040063040902232004007325103439
:100300002AC013840189044023A024001384418956
:10031000044003A104000245731015349240B782D3
:1003200000009382028073A00230A24273A00230C8
:100330004242D2426243F243025492542255B25591
:100340004256D2566257F257064896482649B64951
:10035000464AD64A664BF64B065C965C265DB65D11
:10036000465ED65E665FF65F09617300203000006E
:10037000397101436EC619A0397141536AC866CA02
:1003800062CC5ECE19A0397101535AD056D252D4E4
:100390004ED64AD826DA22DC06DE3301614082825C
:1003A00041114AC026C222C406C68282B24D410112
:1003B000024D924C224CB24B4101024B924A224ACE
:1003C000B2494101024992442244B2404101828033
:1003D0003D432A876373C3029377F700BDEFADE512
:1003E000937606FF3D8ABA960CC34CC30CC74CC724
:1003F0004107E36BD7FE11E28280B306C3408A0651
:100400009702000096966780A6002307B700A30610
:10041000B7002306B700A305B7002305B700A30460
:10042000B7002304B700A303B7002303B700A30258
:10043000B7002302B700A301B7002301B700A30050
:10044000B7002300B700828093F5F50F93968500DF
:10045000D58D93960501D58D61B7939627009702A8
:10046000000096968682E78086FA9680C1171D8FD7
:100470003E96E374C3F8A5B703A581808280EFF2AE
:100480003FF2938781809843050798C3EF10002FB0
:100490003C45FD173CC589E77C413CC5EF10C032A7
:1004A000EF10E05805B70145828001458280014583
:1004B000828001458280EFF2BFEE156495641304DB
:1004C00004689384C46863639400EDBD1C40110408
:1004D0008297D5BFEFF2DFEC156495641304C4680E
:1004E0009384446963639400F1BD1C4011048297B6
:1004F000D5BFEFF2FFEAF93FEF30A026E1B5EFF20A
:100500003FEAB705000037450000D147154793067D
:10051000002001469385254F13058505EF106026C1
:10052000EF10003945B5EFF2BFE7EF10A05DEF2007
:100530009016EF00B02BEF10E056EF005078C13767
:10054000EF10E056012CEF00707A0145A5BDEFF2E7
:100550003FE5D13F0145BDB5EFF2FFE2AA89EF10BB
:10056000E02119C1EF10400A2545EF00F060444139
:100570001304450063968400EF104020014911A840
:10058000138944FF2146CE854A851D2D01E9EF10D0
:10059000E01E19C1EF10A0084A8505B58440D9BFF7
:1005A00009E57D5582807D5531BDEFF27FDF2A84DC
:1005B0002E853289AE844D377DF522852686A54568
:1005C000EF00305E0145231C2401230E0400231D8F
:1005D0000400D9BFEFF2DFDC1E2D41112A84C18B4C
:1005E0009DE71C558DC32EC68297AA84B24501CDC6
:1005F0002A8637450000A28513050506EF009018EE
:1006000026854101C1B31E2C93E707011EAC1E2CA9
:10061000A18B89C73E2CE554A18BFDF35C5489CF97
:1006200022858297AA8405E13E2C93E787003EACA1
:100630005C2C85075CACE9B785679387F7F0FD8D87
:100640002EAC8144D5B7E957E31CF5FAF1BF5C2D18
:1006500085CBEFF2FFD4FD1793F7F70F5CAD2A843B
:10066000014789EF1C5989E70147231D040039A080
:1006700082972A8775D9E957E309F5FE3A8599B338
:100680007D573A858280EFF2BFD1582D09E77D551D
:100690002129014521A05C5999C3829725B3695549
:1006A000C5BFEFF2FFCF582D09E77D55F52E014567
:1006B00021A01C5D99C3829731B36955C5BF0CD188
:1006C00001458280EFF23FCC93894186854A83A71A
:1006D000418663863705EF10E04283A741862A8A68
:1006E000638D370303A441865C4018401309C4FEA0
:1006F0005CC398C340C000C0EF0010717C5099C328
:100700004A8582974A85EF00105B631B55014A8535
:10071000EF00104FEF00B0705285EF10603F71B9DD
:10072000EF00F06F5285EF10A03E4848EF00303ADE
:100730004A85EF00305561BFEFF29FC613840193E5
:10074000130904011C4091C382971104E31C24FF88
:10075000953FEDB7EFF2DFC437060000B745000064
:10076000930800023D4893070020138701948146B7
:1007700013068673938585091385018BEF00F07C42
:100780001385018BEF10C01235B9EFF27FC1411113
:100790002A842E8532C62EC4EF1020083246A24588
:1007A00019C68547630DF6000145410121B958403E
:1007B000938745011CC398CD5CC0C0C9F5B71C40E8
:1007C0006388870083C6550303C7170263FAE600F0
:1007D000D4431387450198C294CDD8C3DCC9E9B787
:1007E0009C43F9BFEFF2DFBB4111B2842E868945ED
:1007F0002A8436C6EF00F03AB246930744011CCC77
:100800005CC846AC14B4014541016DBEEFF2BFB700
:1008100083A7018541112EC62A8491C38297EF10C8
:10082000602E5E2CAA8989CFFD175EACEF10402E9A
:1008300083A7C184014591CB22858297014531A0D0
:10084000B24791E7EF10C02C79554101BDB6EF00DA
:10085000F072232805021034AA85AA8413054401E6
:100860002D37B247635CF0001389C40470008145E2
:100870004A85EF1040184A85EF10E00C4E85EF10C6
:100880002029EF007049885845D5C1B7EFF25FB114
:1008900083A781842A8491C38297EF10A026AA841B
:1008A000484893074401630EF5003115EF00907B33
:1008B00005442685EF10C02519C0EF00F04501451D
:1008C00011B65E2C85075EAC0144E5B7EFF25FAD73
:1008D0004111EF102023138741811C23850793F7D3
:1008E000F70F1CA383A7C18081C72AC68297324510
:1008F000EF1000224101F9B4EFF29FAA4111EF106D
:100900006020138741811C23FD1793F7F70F1CA369
:1009100083A7018181C72AC682973245EF10401F05
:1009200041014DB403C5418182809378080441118F
:10093000639E080091689388482493730801638B31
:1009400003001378E8FF930E000219A891689388BA
:10095000081AE5B713731800930E0003E30503FEAE
:1009600013732800630E0306635806023306C04063
:100970009302D0020A8E814F294F6395E6073373A5
:10098000D6023356D602469303430300850F050E65
:10099000A30F6EFE7DF20DA0137348009302B00208
:1009A0006317030093728800B3325000960279F205
:1009B000930600035480854FFE8663D3FF00BE86F6
:1009C00013781801158F63130804638502006353BD
:1009D000E0007D172A86B308E5001303000221A872
:1009E0008142F1B71373F600118271BF6374B600D0
:1009F0002300660005063388C840E34900FF3A86B5
:100A00006353070001467D173295118F63880200FA
:100A10006374B500230055007D1705056387030245
:100A2000AA96130800031DA86374B6002300D6011C
:100A300005063388C840E34900FF3A866353070040
:100A400001467D173295118FE1BF2A86B308E50074
:100A5000CDB76374B5002300050105053386A640B4
:100A6000E3C9CFFEFD56FD1F6383DF0099E7AA8728
:100A70003306E5001308000231A86376B50033069B
:100A8000F101102210A10505F9BF63F4B70023801E
:100A900007018507B306F640E349D0FE635307001C
:100AA00001473A9541018280EFF29F8F2A849D3D54
:100AB00009C523AC81806FF0FF90EF00304C75D9F1
:100AC00000D9D5BF0D47AA876376C7009377350055
:100AD00091C7AA873E966397C706828093F7F50F62
:100AE00013978700D98F139707015D8FB308C5004F
:100AF000AA87BD463388F84063EB06039357460048
:100B0000C156B386D7029207AA970D48369633830B
:100B1000C700BE86B308D34063621803135726008C
:100B2000F156B306D7020A07BA97369665B798C347
:100B3000D8C398C7C10723AEE7FE6DBF910623AEA9
:100B4000E6FEC9BF8507A38FB7FE71B763F2A504A0
:100B5000B386C500637ED5029345F6FF8147FD1736
:100B60006393F50082803387F6000308070033871C
:100B7000C7002A9723000701DDB73387F5008306F6
:100B800007003307F500850714A3E318F6FE8280FB
:100B90008147E5BF0DC6AA8785050387F5FF850751
:100BA0009306F6FFA38FE7FE09EB3E968507639356
:100BB000C7008280A38F07FED5BF3686F1FE8280F4
:100BC00001476314E600814739A8B307E50083862F
:100BD0000700B387E5009C23B387F640E207E1876F
:100BE00099E30507F9FE3E858280AA8703870700FF
:100BF00001E73385A74082808507CDBFEFF2CFF7AD
:100C00002E89B30B250141112A8CB68563F5AB0003
:100C10001349F5FFFD5BC169374A00006284930AFE
:100C2000B002130B0002FD19130ACA2331A81307DF
:100C300050026389E702637374011CA0130514005A
:100C4000B284138614002A8483070600EDF363063A
:100C50000900637B742F23000400330584414101A4
:100C60006FF00FF501481307D00293063002130509
:100C7000000331A0639E570113684800268683074E
:100C8000160093041600E397E7FE13680801FDB70A
:100C90006395670113688800D5B76395D70013681B
:100CA0000802E9BF6395A70013681800C1BF138746
:100CB00007FDA54663E6E6040147A546294539A098
:100CC0003307A70285043E97130707FD83870400B7
:100CD000138607FDE3F6C6FE038604009306E002D2
:100CE000FD57631FD604838714002546938614009E
:100CF000138507FD6365A60A8147254529433DA065
:100D00009306A0027D57E399D7FC984193042600EF
:100D10009105E35307FC3307E040136808016DBFFA
:100D2000B38767028506B297938707FD038606009F
:100D3000930806FDE37615FF63D307008147B68469
:100D40008386040013068006014593F8B6FF639579
:100D5000C80013F5F60F8504038604009306900679
:100D60006303D60663C5C606930680056303D61CD7
:100D700063C3C604930750026307F61A63757401D0
:100D8000930750021CA08387040013051400638698
:100D9000071A637375011CB0130524005DB51306B3
:100DA000A0026397C7009C4193862400910569B710
:100DB000B684814771B7930630066302D60893065E
:100DC0004006E31DD6FA13682800A94699A09306A9
:100DD00030076303D60C63C5C6029306F0066300B2
:100DE000D61693060007E31BD6F8FD566315D70009
:100DF000136818002147938C4500C14690411DA8F7
:100E000093065007E303D6FC93088007C146E31717
:100E100016F71306C006938C4500E301C5FE1306C2
:100E20008006E31DC5FC904193752800639B051067
:100E300033763601DE852285CD3CE68519B51378FB
:100E4000080163150802BA879306000229A063739C
:100E5000740114A00504FD17E34BF0FE9307F7FFA0
:100E60006343E00005473387E74005079387450064
:100E700063747401944114A013051400229713069F
:100E80000002B306A7406344D000BE855DBB637318
:100E9000750110A10505F5B783AC0500138D45005C
:100EA00063930C00D28C66853EC63AC442C2353B81
:100EB000B247AA86124822476355F00063D3A700C1
:100EC000BE8613780801631E0800BA871306000265
:100ED00031A06373740110A00504BA877D17E3CABB
:100EE000F6FE814763C1D702B68763D30600814708
:100EF0003305F4002A9713060002B307A74063CF17
:100F0000F600EA853DBB3306F40063777601B385CE
:100F1000FC00838505000CA28507E9B763737501A2
:100F200010A10505D9BF6373740110A01305140047
:100F300009BB13680804C146E9BDFD1419B3A146F5
:100F4000C9BD42064186FDB5A38F0BFE39B303A58B
:100F5000C1818280EFF2CFC403A9C181EFF0CFDF5E
:100F600011CD1384C181AA84084019C1EFF02FEE7E
:100F7000930530042685EFF0EFE504C04A856FF055
:100F80006FC48280397126CA2ED232D436D62A86D0
:100F900054109305F007138501B43EDA36C606CE29
:100FA00022CC3AD842DC46DE9139AA8603A5C1811B
:100FB00009E9138501B4F137F2406244D24421615A
:100FC00082802686262D1384C18193E704043EADDA
:100FD0009307F00763F4D7009306F007138601B474
:100FE0008145EFF00FEC1C40A6AFF9B7EFF24FBB15
:100FF000374500001305451B7137374500001305C1
:10100000051C493737470000374500001307471EC6
:101010008D4605468D451305051FAD373745000044
:101020001305052185376FF0EFB931C59166137748
:10103000F50F9386060A09C7BA96882205058280AD
:10104000C167938707F0E98F81CB21851377F50F6F
:101050003697082325058280B707FF00E98F81CBEB
:1010600041859377F50FB697882345058280618186
:10107000369508216505828003A741825C41BA97B5
:101080006305F502B62395E283A60182638FF6001D
:101090009386818290426313F60088C2D44354C180
:1010A000DC43B306E540BA9794C71045B307C700C1
:1010B000630FF500B62381EE938681828C426393A1
:1010C000A5009CC25441D4C35C413E9710C78280A6
:1010D000EFF20FAD83A50183374500001305852589
:1010E000553583A5C183374500001305C526593DF5
:1010F00083A5C182374500001305052861356FF0CF
:101100006FACEFF2EFA913F7C5FFE1462E8663F14E
:10111000E60693073500F19B930687FE63EAF60423
:101120001D8F130687FE23A8C18289665117138479
:101130004182938606EAD8C394C323A407001CC047
:10114000BA9723A0F182C966938606EAB7450000E4
:1011500094C3D8C398C781460546938585311385C6
:1011600001BCEFF02FE8184023A4E1826FF08FA5B7
:10117000AA8537450000130505322935C5BFEFF2B2
:101180002FA239C503A70183130435007198138971
:10119000018381446366870EB1476373F400314471
:1011A000FD55138501BCEFF06FE683A7818283A50F
:1011B00041828328090026853386B740B38688405C
:1011C000138881826368D600138501BCEFF00FECB1
:1011D00081447DA0B384C500BA2003AE440061E71A
:1011E0003307CE40930F47FF63EF8F0A138FC183FE
:1011F000938EC1821303840183260F0083A30E0004
:101200001389C1839382C18263EF6F061307C40001
:101210003297896E3383E500938E0EEA2322C30151
:101220002324C3002320D3010546D8C0B2A003263F
:101230004300B108630416012E9618C61387C60032
:1012400022972320E90063F4E30023A0E20009676A
:10125000130707EA9AA0639A970083A601820147C1
:10126000B22305EE19C32320F800138501BCEFF06B
:10127000EFE183A78183B10481C7A2852685829788
:1012800026856FF02F9405463697B2A02320EF00F5
:10129000E3FFE3FA23A0EE005DBFE385D7FCDC4368
:1012A0000547AE9775BF728631BFEFF26F8F330679
:1012B000B5024111328532C6D9352A8409C5324674
:1012C0008145EFF03F80228541016FF0AF8F45C52A
:1012D000EFF26F8B83A741832A8491C3829783A700
:1012E0004182138941826366F40883A70182637295
:1012F000F408FD55138501BCEFF04FD1835764FF0F
:10130000930944FF81CB035744FF8967938707EA1A
:101310006301F702374500001305C52CA53183563C
:1013200044FF035664FF37450000CE851305852E24
:1013300091398967938707EA231AF4FE938781829C
:101340009843231B04FE63F4E90023A037011387AD
:10135000C1831C43832684FF4E85958F8326090015
:10136000B386D940B6971CC3013B138501BCEFF08F
:10137000EFD16FF08F848280B7070020938607003B
:1013800001479387070021468C426396A5001315F9
:1013900047003E9582800507C106E317C7FE014559
:1013A0008280EFE25FFE2A842E85AE89328AE93799
:1013B0002A89992C83244900930749006390F404F7
:1013C000B92C93E909F8230434012146D2852285FA
:1013D000EFF04FFC83A7018499C322858297EF0029
:1013E0006072032749009307C4005CC358C42322DA
:1013F000F90004C8EF00C0716FE03FFC84407DBF7E
:10140000EFE21FFA83A741842A8491C382972304C1
:101410000400EF00206F544418489307C400D8C25A
:1014200014C31CC85CC4EF00A06E6FE0BFF9EFE20C
:101430009FF52E89AA898937AA84484589332A8449
:101440001DCDD0448145EFF0EFE721462304340160
:10145000A3040400CA852285EFF0CFF383A701849B
:1014600099C322858297EF00E069D8409307C400B2
:1014700091045CC358C49CC004C8EF006069228515
:101480006FE0BFF3EFE2DFF183A741842A8491C3C9
:10149000829723040400EF00E06654441848930741
:1014A000C400D8C214C31CC85CC4EF0060662285A7
:1014B000393D6FE03FF1030585007D8182802390F7
:1014C0000186938701BE13870708DCC39CC3A1076D
:1014D000E39DE7FE3D47238AE18423AC018423A6F4
:1014E000018693874186DCC39CC38280EFE25FEB79
:1014F00003A5C186EFF07FB37D15931735001385E3
:1015000001BE3E9508411307C5FE210523ACE184C9
:10151000EFE01FCB6FE01FEBEFE29FE8EF00805E94
:10152000839701862A89B1E703A5C186EFF0FFAF53
:101530007D1513173500938701BEBA9784439387AF
:10154000818580439385C4FE6305B4028CC383A761
:10155000C185238AA18499C32285829783C741814B
:101560001305C4019385840093F7F70F81EBEFE037
:10157000FFC64A85EF00C0596FE0DFE4EF00A059D5
:10158000CDBFEFE2FFE12A84B52B834744039306E6
:101590004401C19B93E71700230AF40283475403D5
:1015A00013973700938701BEBA97D84314C318CC5A
:1015B000D4C35CC89387C1869443185C558F98C385
:1015C000812B6FE03FE0EFE2BFDD2A84252B184C32
:1015D000544893074401D8C214C35CC81CCC834749
:1015E000540313973700938701BEBA979843631A41
:1015F000F7001387C1861C5C144393C7F7FFF58F70
:101600001CC339236FE01FDCEFE29FD9E5299387E4
:1016100001869A2305079AA3E5296FE0BFDAEFE276
:101620003FD8CD21138701861E23FD17C207C1872E
:101630001EA3634BF00023100700D92983A78185DF
:1016400091C3D93D6FE01FD8E121EDBFEFE25FD537
:1016500003A481854529AA842285B5379147230AA9
:10166000F4021305C404C9242285B1358547631BE0
:10167000F5003C5C81EB2285613326855129693D6B
:101680006FE05FD483A641861307440123A2E1865D
:10169000D8C29387418654C81CCCC5B7EFE25FD04F
:1016A0002A845105411108CC48C80CD050D014D41C
:1016B0003A8658D49305300236853EC642C4EFF0D0
:1016C0006FC0585410544C5008507117B716000092
:1016D0003A969386C664E92EB24722483716000030
:1016E00048CC230BF402A30AF402232C0402814702
:1016F000232204052324040523280402230A0402C8
:10170000232C0406232E04060147A2861306A67284
:10171000A2851305C404E12A83A7018799C3228502
:101720008297014541016FE0FFC9EFE27FC7504951
:10173000144D795718D954C21307450190C218CDDA
:1017400058C98135D13B6FE0FFC7EFE27FC541113A
:10175000B2842E8685452A84368946C03AC63EC460
:1017600042C2EFF01FC4024892472247B2464A865F
:10177000A6852285253741016FE0DFC403A5818559
:101780008280EFE25FC041112E89AA85054532C6ED
:10179000B684BA893E8AEFF09FC92A8411C926858A
:1017A000EFF0FF9D324609E92285EFF0BFCD0144FD
:1017B000228541016FE07FC0AA865288CE872687A6
:1017C000CA852285E13DEDB7EFE29FBD252E83A7B7
:1017D00081850546AA8603C747033D8B631CC70264
:1017E000D04B984F6308E60258C210C303C6570394
:1017F000938647010E06138701BE94CF329750435C
:1018000014C290CF54C3D8CB2126EFF0FFD00145AE
:101810006FE05FBB3685ED2CDDBF83474503054791
:10182000BD8B639FE702EFE2BFB72A84E12C8347B9
:101830004403AA842285C19B93E72700230AF4026C
:10184000EFF07FD81305C404BD2A2685D12483A7D1
:101850008187014581C72285829701456FE09FB648
:101860007D558280834745030947BD8B6390E7041C
:10187000EFE21FB32A8479245448184C930744019B
:10188000AA84D8C214C31CCC5CC81305C404252A7E
:101890002685BD2C2285EFF0DFCE83A74187014549
:1018A00081C72285829701456FE0DFB17D55828037
:1018B000EFE21FAF8346650305473317D70018DDF6
:1018C0000947A30AD502230AE502693F83A7818558
:1018D00099C3EFF07FC401456FE0DFAE5449184D66
:1018E00093074501D8C214C31CCD5CC98280EFE2C6
:1018F0003FAB4111B2842E86A9452A8436C63AC42C
:101900003EC2EFF01FAA9247B2462247F99B1CB491
:101910009307440144CC14D02324040258D01CCC97
:101920005CC841016FE01FAAEFE29FA72A84D92A71
:10193000AA84228565372685E12A2285EFF05FACEF
:1019400001456FE03FA8EFE2BFA52A84652AAA847B
:10195000228569371C342685F99B1CB4552A83A738
:10196000C18499C322858297EFE01FB15C503E95F8
:1019700008D4492A13878188032847003706008046
:10198000938781881346E6FF98436315F802938690
:10199000C1879042050690C29306440154C358C8BB
:1019A00094C31CCC1C3493E717001CB4952201454A
:1019B0006FE05FA1544B0C546385B6008D8EE378C5
:1019C000D6FCBA87D1B71C35858B85C7EFE25F9D02
:1019D00083A781842A8491C382972D22AA84228599
:1019E000F53D268535221C340145F99B1CB46FE07A
:1019F0007F9D7D55828085476381F50263C5B70071
:101A000085C1014582808947638FF5008D47E39A40
:101A1000F5FE1C3593E7270009A85C511CC2D5B719
:101A20001C425CD1F9BF1C35F59B1CB5D9BFEFE258
:101A3000BF94EFE07FA42A8CF120B70900802A8AA6
:101A40009384818893C9E9FF8D4B8040631694008D
:101A500052857D286FE0DF9548481309C4FE3305A1
:101A6000AC40E3E7A9FE83A7018899C34A85829722
:101A70004A85EFF0BFE61C4448448297EFE0DF9FC1
:101A800083A741882A8C99C34A858297834754FF4C
:101A900013F7E70FA30AE4FE8D8BE39877FB4A85E3
:101AA0005D3565B793878188DCC39CC38280828063
:101AB0001106719A2A8837C7ADDE130506F8AA8782
:101AC0001307F7EE631EF600A167938707882322AA
:101AD000D6F82324B6FA232006F92324F6F88280C8
:101AE00098C39107C5B737F700E01C43B7060080DD
:101AF000D58F1CC3828037F700E01C43860785839F
:101B00001CC3828021651305058073150530828012
:101B1000731005308280EFE2BF88138781891843F4
:101B20009387818919E323A8A18823AAB18805474F
:101B300098C3553F6FE01F892A8781471843631474
:101B4000A7003E8582808507D5BFB707EFBE37E780
:101B500000E0938707083CC701458280EFE25F847D
:101B6000374500001305C535EFF0CFC101456FE0E3
:101B70007F85EFE2FF822A84FD54375900007D14EF
:101B8000631494006FE01F84130549ACEFF08FBF1E
:101B9000FDB7EFE24FFF0041AA8437590000B75963
:101BA0000000631494006FE05F819305C4FE130589
:101BB00089ACEFF02FBD1C40638697001385C9AC3C
:101BC000EFF04FBC0040F1BFEFE28FFD2E89EFF048
:101BD000CF812A84EFF05FA383240900639C240152
:101BE000EFF0FFA3A14763C3870011E021442285E2
:101BF0006FE04FFD138544FFEFE03FFF6353A40008
:101C00002A848440E1BFEFE22FF70545EFF0CFF6DD
:101C1000B7490000130945002A84CA851385096164
:101C20006537AA85AA843745000013860961130524
:101C30008561EFF02FB526852D3F37450000130550
:101C4000C565EFF02FB44040B7490000054A894A06
:101C5000374B0000B74B0000374C0000B74C00007A
:101C6000374D00006315890001456FE06FF40347AD
:101C700094021385C969930644FF2146A685EFF0B7
:101C80006FB08347840213858C6ABD8B638E4701D6
:101C900013054C6B638A570113850B6C91C7114771
:101CA0006396E7001305CB6CEFF0CFAD4C4C930778
:101CB0003002AE8698226306F70210509307400662
:101CC0000848B295B386D540B386F602585C5C509E
:101CD000898D13058D6DB3D6C602EFF0AFAA004013
:101CE00051B78506C1BFEFE20FEA41110945EFF098
:101CF000AFE893094500374900002A84CE851305D3
:101D0000095BEFF07FECAA85AA8437450000130633
:101D1000095B1305C55BEFF0EFA62685EFF07FE5C5
:101D2000374500001305855DEFF0CFA54040374AE9
:101D30000000B74A0000375B000063968900014548
:101D400041016FE08FE71A281C44930644FF1309F2
:101D5000840036C63AC44A856306F902EFF0DFDD37
:101D60002247B246AA872146A68513850A5FEFF06F
:101D70006FA14A85EFF0FFE113058B52EFF08FA0C2
:101D8000004065BFEFF05FDB2247B246AA872146DD
:101D9000A68513050A60EFF0EF9EDDB7EFE2AFDE38
:101DA00041111145EFF04FDD93094500374900001F
:101DB0002A84CE851305493FEFF01FE1AA85AA8446
:101DC000374500001306493F1305C53FEFF08F9BD1
:101DD0002685EFF01FDA3745000013050542EFF0C6
:101DE0006F9A4040374A0000B74A0000375B000056
:101DF00063968900014541016FE02FDC1C44130903
:101E00008400930644FF18486309F9024A8536C6E0
:101E10003AC4EFF07FD22247B246AA872146A68570
:101E200013850A44EFF00F964A85EFF09FD613050D
:101E30008B52EFF02F95004065BF2146A685130514
:101E40008A45EFF02F94C5BFEFE2EFD341110D4566
:101E5000EFF08FD2B7490000130945002A84CA85E4
:101E60001385C954EFF05FD6AA85AA8437450000D0
:101E70001386C95413054555EFF0CF902685EFF032
:101E80005FCF3745000013058557EFF0AF8F404017
:101E9000B749000063168900014541016FE0EFD1A9
:101EA000930644FF1305840036C6EFF0FFC80348CD
:101EB00034015C48B246AA8821472146A68513858D
:101EC0008959EFF02F8C0040F1B7EFE2CFCB4111F1
:101ED0001545EFF06FCA93094500374900002A8481
:101EE000CE851305C946EFF03FCEAA85AA843745B3
:101EF00000001306C94613054547EFF0AF88268555
:101F0000EFF03FC73745000013058549EFF08F8795
:101F10004040374A0000B74A0000375B0000639634
:101F20008900014541016FE04FC97A285E281044BD
:101F3000930644FF1309840036C63AC43EC24A855C
:101F40006307C902EFF05FBF92472247B2462A8873
:101F50002146A68513854A4BEFF0CF824A85EFF0E4
:101F60005FC313058B52EFF0EF8100404DBFEFF0E0
:101F7000BFBC92472247B2462A882146A685130550
:101F8000CA4CEFF02F80D5B7EFE2EFBF41111945F2
:101F9000EFF08FBE93094500374900002A84CE85B3
:101FA0001305494EEFF05FC2AA85AA8437450000A9
:101FB0001306494E1305054FEFE0DFFC2685EFF0D1
:101FC0005FBB374500001305C550EFE0BFFB404045
:101FD000374A0000B74A0000375B0000639689006B
:101FE000014541016FE06FBD1A2C1C44930644FF6C
:101FF0001309840036C63AC44A856306F902EFF035
:10200000BFB32247B246AA872146A68513854A5206
:10201000EFE05FF74A85EFF0DFB713058B52EFE093
:102020007FF6004065BFEFF03FB12247B246AA8776
:102030002146A68513058A53EFE0DFF4DDB7EFE212
:102040008FB45D712545EFF02FB391651306000540
:102050002A8413094500938585000A85EF101069CD
:10206000B7490000CA851385C938EFF0FFB5AA85C6
:10207000AA84374500001386C93813054539EFE0B7
:102080007FF02685EFF0FFAE374500001305C53B16
:10209000EFE05FEF4040D149374A00006316890006
:1020A000014561616FE06FB11C44930644FF63E03A
:1020B000F90298088A07BA9703A707FB1C2821464C
:1020C000A68513050A3EEFE0FFEB0040C1BF46477F
:1020D000F5B7EFE24FAB2945EFF00FAAB749000083
:1020E000130945002A84CA8513850970EFF0DFAD16
:1020F000AA85AA84374500001386097013058570E8
:10210000EFE05FE82685EFF0DFA637450000130516
:102110000573EFE03FE74040B7490000374A000051
:10212000B74A0000631E8900EFE00FB5AA85374566
:10213000000013058578EFE0FFE401456FE0EFA7AD
:102140005C4C184C13854975930644FF2146A685BF
:10215000EFE05FE38347D4FF1385CA76858B99E36D
:1021600013058A77EFE01FE200406DBFEFE2AFA1F9
:102170003745000013054536EFE0DFE003A4018A90
:10218000B7490000374A000083A7418A6365F4001D
:1021900001456FE08FA20440094693858937268563
:1021A000EF10F06319C55040A6851305CA37EFE05C
:1021B0007FDD3104D1BFEFE20F9D375500001305DD
:1021C00085C2EFE03FDC03A4018AB7590000375A0B
:1021D000000083A7418A636BF400375500001305A4
:1021E0008552EFE03FDA01456FE02F9D044019462C
:1021F000938549C42685EF10905E01E95040938590
:1022000064001305CAC4EFE0FFD73104D9B7054510
:102210008280EFE24F9779712A84AA959306000293
:10222000254783070400B38485406385D70A638309
:10223000E70A0145638B0410014913070002A54614
:10224000B307240183870700638AE7086388D708F8
:102250006314990883A9018A83AA418A375B000025
:1022600063F0590903AA0900194693054BC4528526
:10227000EF10F05659E54A86A28513056A00EF1063
:10228000105641E14A9A83076A00A5EF83A98900A5
:10229000638809041306800281452800EFE04F930C
:1022A00013098100CA86A28701450147130800026D
:1022B000A548294313062002130EC0058385070095
:1022C0006384050163961505631F9702A94763039D
:1022D000F50469A80504B1B705099DB7E31C09F623
:1022E000A287038707001377F7FD79E737550000CA
:1022F000130505C123800700A285EFE0BFC87D5507
:10230000A9A0B109B1BF23800700050785077DB7E4
:1023100063106504375500001305C5BEEFE09FC686
:102320000018B7540000832509001385C4C01109A3
:10233000EFE05FC5E31989FE3755000013058552AC
:10234000EFE05FC429452C00829945616FE0EF867C
:10235000637E970005056392C504850705079CC247
:10236000838507006381C5026364970069FD8DBFA3
:10237000838E17006396C5016394CE008507050719
:1023800085070507F1BFE37397FE23800700050764
:1023900085079106E36497F2D1BF9CC2838507004D
:1023A0006389050163871501E30297FC850705072B
:1023B000F5B7E36097FE5DBF850725B7EFD2DFFB7A
:1023C0008307050099E781450145EFF0DFDE6FD017
:1023D0003FFE03AA018AAA8981440149375B0000B4
:1023E000B75B000083A7418A6369FA00EDD04A8693
:1023F000A6854E85EFE00FFAD9BF03240A001946DF
:1024000093054BC42285EF10903D21E14E85EF10DE
:10241000F03B19042A86A2854E85EF10503C15E545
:10242000631709002285EF10703A2A89A284A687D3
:1024300022870386070001EE858F63D327013E893B
:10244000A28513854BC5EFE0FFB3310A61BF830658
:102450000700FDD2E312D6FE85070507D9BFEFD2EC
:102460003FF4EFF04FFA01456FD0DFF5EFD25FF3A5
:10247000EFE01FC601456FD0FFF4EFD27FF203A556
:10248000C189EFE0AFC001456FD0DFF3EFD25FF15C
:10249000B75700009387C75223A0F18AB7570000AF
:1024A0009387C76723A2F18AB75700009387C7674E
:1024B00023A4F18AB75700009387C76793050021CB
:1024C000054523A6F18A1384C189EFE01FDE08C009
:1024D00019E937550000130585D0EFE0BFAA7D54F8
:1024E00022856FD03FEEB725000037550000A94781
:1024F0002D479306004001469385C560130505D21C
:10250000EFF02FA8AA840840B75500008146014685
:10251000938585D2EFE00FAD0144F9D02685EFF029
:102520002FB97DBFEFD2DFE7EFF07FCE0DC5B755F6
:102530000000938545CD138501C6EF103028B755AF
:102540000000938545CE138501C6EF1050251385F5
:1025500001C66FD03FE7B75500009385C5CDE1BFF9
:10256000EFD21FE42A8437550000130545D4EFE06D
:102570007FA1EFF03FFBAA85375500001306A41B8F
:102580001305C5D4EFE01FA001456FD0BFE3EFD224
:102590003FE141112AC6EFD03FFCB24511E9375562
:1025A0000000130585CEEFE0FF9D41016FD09FE154
:1025B00083A7C189AA841384C18983A7C720E3861E
:1025C000A7FE93053014EFE0EF8065F11C4003A5F2
:1025D000C72009C9EFE0AF871C40814503A5C7208C
:1025E000EFE0EF8D00401306000581451305A41BA5
:1025F000EFD01FDEB72500002315042023269420EA
:102600009385A5472685EFE08F8B45B7EFD25FD640
:1026100083A7C18941119384C18903C74702136706
:1026200017002382E70283A7C72091E7EFE03F92DC
:1026300019C1EFF0DFF5EFF0FFEEEFE0BF94375B8D
:102640000000B75B0000B7590000375A0000B75AC6
:102650000000375C0000B75C00009C408546130614
:10266000F10003A5C720FD55EFE0EF818547631A10
:10267000F5000309F100ED4780406319F90008D027
:10268000E9BF8840FD55EFE06F98C1BF1C506392D1
:10269000A7029307B0056315F90089471CD075BFE1
:1026A00023200402E30B09FAA5476314F912014938
:1026B000D1A80947E398E7FE2320040293071004FA
:1026C0006312F9046E30D1D9FD15C205C1816EB017
:1026D0009307A41B13070005B385E5021306000545
:1026E0003E859385A502A295EF105000EF10100EC5
:1026F0001375F50F2305A420A305A4202285EFF070
:102700003FE6A1BF930720046311F90216347E301F
:102710001387F6FF63D8E70085077EB09307A41BF5
:102720006E304DBF9DDA7AB0D5BF93074004631079
:10273000F9028347B42095D3138509D3EFE09F8432
:1027400098408347B720FD17A305F72039B79307B3
:102750003004E319F9F48347B4200347A420E3FECF
:10276000E7EE3E948305A41B13854AD3EFE09F81D7
:1027700098408347B7208507C1BF138509D3EFE091
:102780007F80050980408347B420E348F9FE1305A4
:102790008A52EFE02FFFEFF09FA785471304A41B99
:1027A0006315F5002285EFF07FC1EFF0BFD72286D9
:1027B000AA851385CCD4EFE0EFFC80401305A41B61
:1027C000EF10D0001375F50F2305A420A305A42056
:1027D00069B59307F0076305F900A1476315F90888
:1027E0008347B420E38B07E60346A420FD1793F745
:1027F000F70F7D161376F60F2305C420A305F420EA
:1028000063F8C7049385B71B1385A71B1D8EA2957C
:102810002295EFE0AFB39C4013858BD303C7A7206D
:102820003E97230D071A83C5B7209385A51BBE9538
:10283000EFE04FF59C4003C4B7209C4083C7A7201E
:10284000E3CD87E0138509D3EFE0CFF30504F5B7B7
:1028500013050BD4EFE00FF39C4003C7A720BA97F2
:10286000238D071ADDBB35478347A4206305E900A4
:102870002947631EE90EB9CB035984029147130D12
:10288000A41B63FB2709930DA41613060005EA8514
:102890006E85EF1060631DC91309A4024A851309F0
:1028A000090513060005CA85EF104064E3982DFF63
:1028B0001306000581456E85EFD09FB10346A42025
:1028C000EA856E85EF10806295471EB41E347EB097
:1028D000EFF0FF9385476312F5029C4083C74702E0
:1028E000858B89C713058A52EFE0CFE9884083457D
:1028F000A5201305A51BEFF0DF91EFF0BFC2EFE0BD
:102900006FE880401306000581451305A41BEFD036
:102910003FAC2315042091B3630109021305F9FFAD
:10292000930700053305F50213060005EA85130534
:10293000A5022295EF10405951D9930D000533059A
:10294000B9031306000581451305A5022295EFD0B2
:102950003FA80A340346A420EA853305B5031305CE
:10296000A5022295EF1080581E348507B9BF1307C2
:10297000F0046374F700230504200346B420834762
:10298000A4206370F6089305A61B1305B61BA29539
:102990003386C7402295EFE06F9B8C4083C7B520FC
:1029A0003387F500230D271B03C74502058B01CB99
:1029B0009387A71BBE9513058CACEFE0AFDC9C4062
:1029C00003C4B7209C4083C7A7206346F402984005
:1029D0008347A7208346B7208507850693F7F70F1F
:1029E000A305D7202305F7209306F004E3F7F6C6E6
:1029F000231507209DB1138509D3EFE0AFD8050457
:102A0000D1B7A297238D271B83474402858BE1D33F
:102A1000CA8513854AD3EFE0EFD655BF7C41232802
:102A20000504232A05049C4381CBEFD27F979305AD
:102A3000850482976FD01F9901458280EFD2BF94A1
:102A400036899DCAAA843284B309D600294A1C203B
:102A5000639B4701BE2C93F7070491C7FC40B54523
:102A600026859C478297FC408305040026859C4769
:102A700005048297E31D34FD4A856FD01F94EFD281
:102A80003F9293F705102A8491C71A2D6155137749
:102A9000071035CF13F7054011C71A2C615513776E
:102AA000074035C713F705049304000401E7262CFB
:102AB00093F40404384893F5F50F2EAC39EBA1C715
:102AC00068442981420541813105EFE04FEB7044B4
:102AD0002A89310529824206418281452320A900A5
:102AE000EFD05FFE232209003E2C23240900232877
:102AF000240593E707103EAC7C4013060010C14547
:102B0000DC43228582973E2C0145DD8C26AC6FD0BC
:102B10007F8BF5DB93E505102EACF5B70948AA8746
:102B200063810503EFD2DF870D4863820503054704
:102B30006399E5041A2D1377F7FD1AAD01456FD09F
:102B40007F881A2D136707021AAD014582803287EC
:102B500075D6504274454C2D2982A9824206C20680
:102B60004182C1826304D6001D45F1F91443B4C704
:102B70005443F4C7E1D5F443BA853E859442829626
:102B800075BF7C41DC4382975DBFEFD2CFFF3684B7
:102B9000B1CA3E2DAA89328993F70710B6849DE306
:102BA0007D5AA94A83A749044E85DC478297630969
:102BB00045012300A900FD14050963035501FDF03B
:102BC000058C0DA02449368A854AEFE0BFF3FE202C
:102BD000DA202A869444631AF70081EAEFE05FF373
:102BE0003304444122856FD04FFD98403E97034BFC
:102BF000070003A7C9048507C2072983C1834207C9
:102C0000FEA0418363E4E70023930400639456012C
:102C100023A404003285EFE0BFEF7D1A2300690191
:102C20000509E3140AFA6DBF582D854763ECE702E6
:102C30003E2D93F707109DC7EFD28FF62A842849BF
:102C4000EFE0EFE83E2C232804041306001093F76E
:102C5000F7EF3EAC7C40C5452285DC4382970145B9
:102C60006FD04FF601458280EFD28FF337370000E7
:102C70001307C7A118D5373700001307E7A758D5A2
:102C800037370000130787C218D9373700001307FA
:102C9000A7B858D9373700001307C7A318DD37374F
:102CA00000001307C7B1420658DD34C14182232A10
:102CB00005002320050223220502EFD07F8E6FD06E
:102CC0006FF093F5F50F85476391F50AEFD2AFEBFF
:102CD00020494111AA847D598549FC402685DC475D
:102CE00082972A8A63072505EFE0DFE15A201C401E
:102CF000BA97238047015E20F8448507C2072983DD
:102D0000C18342075EA0418363E4E700231204000D
:102D100076205E20639CD7008507C207C1837EA012
:102D20002324340163E4E70023130400EFE05FDEB3
:102D30006DB79C5085C3EFE0FFDC5A206E20636EB8
:102D4000B700B305B7402EC6EFE09FDC9C50B245FC
:102D50002685829741016FD04FE6FC44998DA98367
:102D6000C207C183B385B740F9BF828001CEEFD2DD
:102D70002FE37841B2878E23184332220297014510
:102D80006FD04FE47D558280EFD28FE1138741CE23
:102D900078432E86AA851843138541CE02976FD0BB
:102DA0006FE2EFD2EFDF138741CE78432E86AA85FC
:102DB0005843138541CE02976FD0CFE0EFD24FDE5C
:102DC000138741CE7843AA85138541CE18470297D1
:102DD0006FD04FDF05C611476392E602EFD24FDC9A
:102DE0007C410E2241119C4736C632C4829722464E
:102DF000B2462AA2368541016FD0CFDC81463685A6
:102E000082801DC2B28711466390C602EFD24FD9AD
:102E10007841B2238E235843411136C60297B246F9
:102E2000410136856FD00FDA814636858280EFD238
:102E30002FD7938741CE4947D8CB373700001307A8
:102E400047DDD8DB37370000130727E098DF373737
:102E500000001307C7D6ECC3B0C3AA850D4613857F
:102E600041CE23A0070223A2070223A4070223A620
:102E7000070223A80702D8DFEFD08FF201456FD0F9
:102E80006FD4370500201305C568828037150020F0
:102E90001305C5688280EFD2AFD0B707002003A723
:102EA00007169307803EC1563357F702B7E700E095
:102EB0002386D7402387D740856623A0D710916605
:102EC00023A0D710B7F700E023A0070023A2070034
:102ED000014690C78146D4C781461306F7FF90CBC1
:102EE000D4CB3D4798C3EFD00FDDEFF09FF92A8494
:102EF000EFF0DFF9AA852285EFE0AFA0375500009B
:102F0000130545DCEFE00F856FD0CFCB7311013493
:102F1000EFD0DF9BB7F700E023A20700EFD02FD65A
:102F2000EFD09F9D73110134730020308147854697
:102F3000130700023396F6006306A6008507E39B9D
:102F4000E7FEFD573E858280EFD28FC5854513058C
:102F50000002EF0030626FD0EFC6EFD26FC485453C
:102F60002145EF0030616FD0EFC5EFD26FC38545CB
:102F70001145EF0030606FD0EFC4EFD26FC28545CE
:102F80004145EF00305F6FD0EFC3EFD26FC1854591
:102F900013050004EF00105E6FD0CFC2EFD24FC018
:102FA00095653755000001469385C5DC1305454BF3
:102FB000EFF0FFE76FD00FC19307400663ECA70067
:102FC000931745001565130545E63E951841FD57D5
:102FD0006313F70001458280EFD28FBC411113F5D6
:102FE000F50F32C6EFF05FFD11C54E25324608459C
:102FF000EF00903D41016FD0EFBCEFD26FBA13F5F7
:10300000F50FEFF07FFBAA87014589C7CE278847D8
:10301000EF00F03A6FD00FBBEFD28FB8011113F56C
:10302000F50F3284EFF05FF905C55C412AC682973F
:1030300032455C45FC82C1473ECE8D473ECC09C43B
:103040001547631AE40002CE08454C08EF00302B08
:1030500005616FD02FB705476315E40091473ECE59
:10306000E5B76315F40093078002D5BF8947631560
:10307000F40093078004E5B791476314F400D14747
:10308000F9BF99476314F400F147D1BF9D47E31D91
:10309000F4FAE147E9B7EFD20FAF13F5F50FAE84BD
:1030A000B289368A3A89EFF03FF1994731CD4845E8
:1030B000EFF0DFE73D472A8499476367A704EFE015
:1030C0007FA4B146B306D402B707002013870708D0
:1030D0002A8693870708369783160700639F960012
:1030E0004C43639C45012E236399350118476316B1
:1030F0002701EFE0FFA1814701A87D576389E60022
:103100003285EFE0FFA09D473E856FD00FAB314584
:103110003305A4023E9506A1232245012311350162
:10312000232425013285F1B7EFD28FA713F5F50FD0
:10313000EFF09FE819471DC94845EFF03FDFBD4755
:103140002A84194763E4A702EFE0DF9BB147330409
:10315000F402B7070020938707087D57A29783964C
:1031600007006398E600EFE0BF9A01473A856FD009
:103170006FA541677D1798C323A2070023A407000A
:10318000DDB7EFD24FA0011113F5F50F328AEFF042
:10319000BFE2994721C185442A8463159A104845A6
:1031A000EFF0DFD83D47AA8499476365A702EFE0B7
:1031B0007F95B14AB38754033709002013090908E2
:1031C000AA893E9903170900FD576319F700EFE03C
:1031D0003F9499473E8505616FD02F9E5C40829752
:1031E00085450545EF0010395C440D473AC47C82A3
:1031F0003EC88357290002CA52CE638C4709C1C713
:103200000947638DE70808444C00EF00500F18444D
:10321000B7170140938607C005456302D7020945E9
:10322000630FF700938707400D45630AF700B72740
:1032300001409387078001456313F700114593F51B
:10324000F40FEF0010190808EF00500295679387FC
:1032500047DE8E04BE94D04037E700E093060005B9
:10326000B307C7002380D7409357560093870704BE
:1032700085468A07B396C600BA9794C34E85EFE099
:103280003F89814781BF930780023EC6A1473ECC5C
:103290009DBF930780043EC656CCB5B791473EC646
:1032A000C147F5B79947E3170AF24845EFF01FC841
:1032B0003D479947E360A7F293173500156513055D
:1032C00045DE3E9558419357570093870706B394C0
:1032D000E4008A0737E700E0BA9784C35DB7EFD20E
:1032E0002F8CEFF0BFC4B1473305F502B7070020BC
:1032F000938707083E955C4199C3084582976FD034
:103300006F8C73110134EFD06FDC0545EF00A07CAA
:1033100019C50545EFF0BFFC0545EF00A07DEFD0D6
:10332000AFDD731101347300203073110134EFD01D
:10333000EFD90945EF00207A19C50945EFF03FFAAA
:103340000945EF00207BEFD02FDB731101347300B0
:10335000203073110134EFD06FD71145EF00A07703
:1033600019C51145EFF0BFF71145EF00A078EFD078
:10337000AFD8731101347300203073110134EFD0D2
:10338000EFD42145EF00207519C52145EFF03FF539
:103390002145EF002076EFD02FD673110134730052
:1033A000203073110134EFD06FD24145EF00A0728D
:1033B00019C54145EFF0BFF24145EF00A073EFD0D2
:1033C000AFD3731101347300203073110134EFD087
:1033D000EFCF13050002EF0000701DCD13050002B2
:1033E000EFF0FFEF13050004EFF07FEF1305000887
:1033F000EFF0FFEE13050010EFF07FEE1305002055
:10340000EFF0FFED1305003EEF00C06EEFD0CFCE22
:10341000731101347300203013050004EF00A06B1A
:1034200055FD13050008452D55F9130500106525B8
:1034300055F513050020452555F1C9BF7311013419
:10344000EFD0CFC813050040792521C113050040F6
:10345000EFF0FFE8056513050580EFF05FE805650F
:10346000EFF0FFE70965EFF09FE71165EFF03FE749
:103470002165EFF0DFE64165130505C0A52DEFD00E
:10348000AFC7731101347300203005651305058043
:1034900099254DFD0565812555F909652D2D5DF5AC
:1034A0001165152D45F521653D254DF1C9BF014536
:1034B0008280EFC2FFEE9C412041A14641111CC019
:1034C000B1473EA4DC412316040013F7F700630163
:1034D000D702A546631ED70005675AA013D7470039
:1034E0000D8B01C785466308D7002313040031A064
:1034F00023120400E5B709677AA099838D8B0547ED
:103500006389E70081C709476387E706231404003E
:1035100021A0930700601EA41848B7470140938775
:1035200007806316F704116585451105EF009004C7
:1035300093070020B71401407C820D49E1474C00FD
:10354000138504803EC64AC45D2B930700407C82ED
:103550004C009147138504803EC64AC44D23084859
:10356000A285EF00100308488545EF00900B014548
:1035700041016FC03FE59307004071BFEFC2BFE05C
:10358000B71400201384446E930750035CC83719A6
:103590000020B74701401306C96893870780744627
:1035A0001CC895679387874B7CC2B70700C0F58F0F
:1035B000C166A106716713070720D58F11654111F8
:1035C00038C67CC68545B7070C00110518C01CC459
:1035D0002322040023160400EF00C079B71901402C
:1035E000930700207C820D4AE1474C001385098037
:1035F00052C43EC62923930700407C824C00914769
:10360000138509803EC652C4DD2908489385446E5F
:10361000EF00207808488545EF00B000B75500005E
:103620009386446E13063010938545DC1305C968F4
:10363000EFF08FE3014541016FC03FD8EFC25FD685
:103640002041930500020848EF00700219C51C488C
:10365000CA231375F50F6FC0FFD67D55EDBFEFC2BE
:103660003FD424412E84884893050004EF003000A5
:103670007DD99C4842044180C2A305456FC09FD4B8
:10368000EFC21FD2C1473841638AF502C547639430
:10369000F502544B054693D7560093870706331619
:1036A000D6008A07B7E600E0B69790C30146084BFC
:1036B00093055052512701456FC0DFD0544B05464A
:1036C00093D75600938707043316D6008A07B7E6C8
:1036D00000E0B69790C30546D9BF411122C626C463
:1036E00073110134B7140020EFD04F9E9387C46844
:1036F000A043930550520848412719C985451385B1
:10370000C468EFF00FDC084893055052EF00807A50
:10371000EFD08F9E731101343244A24441017300F3
:10372000203073110134EFD06F9A37550000130524
:10373000854DEFD03F85EFD02F9C7311013473007E
:10374000203073110134EFD06F9837550000130506
:10375000C54CEFD03F83EFD02F9A73110134730023
:103760002030EFC2FFC3375500001305854EEFD060
:103770007F813D22B707002083A50716375500003B
:103780001305C54FEFD01F80E92CAA8537550000DF
:103790001305C550EFD00FFF375500001305C55175
:1037A000EFD04FFE01A0B71702409843B706FFF0D5
:1037B00041111367170098C3D84337060200758F6D
:1037C000D8C39843B706F7FEFD16758F98C3984384
:1037D000B706FCFFFD16758F98C3D843B70601FFE7
:1037E000FD16758FD8C39843B70600ECFD16758F8C
:1037F00098C33707FF0098C723A6070202C402C672
:103800009843C166558F98C3B716024005679C421E
:10381000F18F3EC6A24785073EC4B24781E7A24763
:10382000E397E7FEB71702409C431397E7006357FF
:10383000070685473EC632478547631FF704B7171B
:103840000240D843B706C1FFFD16D8C3D843D8C33A
:10385000D84313670740D8C3D843758FD8C3D8431C
:10386000B7062900558FD8C39843B7060001558F76
:1038700098C3984393166700E3DD06FED843B71656
:103880000240719BD8C3D84313672700D8C3214790
:10389000DC42B18BE39EE7FE4101828002C661BF3C
:1038A000B7160240D842B70700201146318B9387E4
:1038B00007166305C70021466308C70237177A0059
:1038C0001307072098C33717024058431183937694
:1038D000F70037070020130707143697142398437F
:1038E0003357D70098C38280D842D4424166498377
:1038F0003D8BF18E1306270015CF3D47630FE6027F
:103900004147630FE602454781456313E6004146A0
:10391000A1E23747024003270780418B0DC73717C5
:103920007A00130707203306C70290C3C9DD984306
:10393000058349BF81454946E1BF85453546C9BF35
:1039400081453D46F1B737173D0013070790E1BFAA
:103950003715024058559316F700585563DF060493
:1039600011833D8B9306170037177A001307072042
:103970003357D70298C35455A182BD8A8DE295462C
:103980003307D702058398C337170240585794432B
:103990003D8B050733D7E60298C3984369B70545C1
:1039A0006394A600E546E9BF3D456396A600D1466F
:1039B0003387E602C9BF8906E5BF3D8B9306170032
:1039C00037177A00130707203357D702F1B701A042
:1039D0007390123497D1FF1F9381C1F817C1002053
:1039E0001301416217250000130545CB97C5FF1F42
:1039F000938545611386818063FAC50083220500A3
:103A000023A0550011059105E3EAC5FE13858180C9
:103A100097E5FF1F9385C5CE6377B500232005008A
:103A20001105E36DB5FEFD42739002BCFD4273903B
:103A30004280B7820000938202807390023097C266
:103A4000FFFF9382625C93E2320073905230EFF09A
:103A50009FD597D2FFFF9382C2AF73901234730049
:103A60002030B7F7FF1F03A5477082805841032815
:103A700005004C4537060140930706403E979346A4
:103A8000F8FFB1C583250640F58D2320B640D0430D
:103A9000F18ED4C31443B3E6060114C31841904712
:103AA0009346F7FF758E90C7D047F18ED4C7144563
:103AB00041466399C6009447D98E94C7D447558F21
:103AC000D8C78280B6979443558F98C382801C4391
:103AD000F58F1CC38280B70701401387074083A777
:103AE0000740584B698F09C77D8D3335A000828010
:103AF00001458280B707014023AAA74082809C45E8
:103B000013F7070113F8F70001C7D8413368E8003D
:103B10008E2113F7F50F39C318418146854E3D4F6D
:103B2000930F800293028004214E3396DE00B3F897
:103B3000C500631116039398260033131F01134326
:103B4000F3FF3377E300B318180133E7E800639F0E
:103B5000F70550C98506E39AC6FD18C11307F00F93
:103B60006375B70454412146854E3D4F930F800243
:103B700093028004414EB398CE0033F7150163924F
:103B8000E8021317260001173313EF001343F3FF66
:103B9000B376D3003317E800D98E639DF701232A4B
:103BA00015010506E319C6FD54C18280E39457FA56
:103BB00010C94DB7E39757FE23281501DDB7084517
:103BC0006D8D3335A000828019C20CC982804CC92A
:103BD000828013F7C50F93F73500B7050140BA95FA
:103BE00094458A073D473317F7001347F7FF758F52
:103BF00098C598453315F500598D88C582803717CB
:103C000002405C439146B18B6385D700A146638235
:103C1000D706B7177A00938707201CC137160240D2
:103C20005C4237070020130707159183BD8BBA97B5
:103C300094231C41B3D7D7005CC15442A1829D8A12
:103C4000BA969422B3D6D70014C55442AD829D8A49
:103C500036971823B3D7E7005CC55842398393766B
:103C600037001387418036971823B3D7E7021CC962
:103C700082805C435843C166C983758FB7F6FF1FC6
:103C800083A6C670BD8B890713961601634806008C
:103C9000C54601466392D702C94739A88946638F52
:103CA000D702BD46638ED702C146638ED702C54692
:103CB00001466393D700C1471DEF374702400327F2
:103CC0000780418B05C737177A0013070720B30712
:103CD000F7021CC121D61C41858381B701466DBF07
:103CE0000546B547D1BF0146BD47F9B737173D0077
:103CF00013070790E9BFB7150240D8559316F70090
:103D0000D85563DF060411833D8B930617003717E0
:103D10007A00130707203357D70218C1D455A18260
:103D2000BD8A8DE295463307D702058318C1371740
:103D30000240585714413D8B050733D7E60218C19E
:103D4000184171B785456394B600E546E9BFBD45A6
:103D50006396B600D1463387E602C9BF8906E5BF40
:103D60003D8B9306170037177A0013070720335748
:103D7000D702F1B799C5371702401C4F5D8D08CFA8
:103D80008280B7170240984F1345F5FF798D88CF91
:103D90008280EFC2EFE01629F577FD17F58FF62147
:103DA000DA257971D58F1EA95625FD779387379F20
:103DB000F58FD6212A842EC6D58F9625D58FB62588
:103DC000D58F5EA55E29C207C18393F7F7CFD98F40
:103DD0005EA96808EFF0BFE2B7470140938707800C
:103DE000B245631EF402A2576547B387E7029841C4
:103DF000930640060A07B3D7E70233D7D702B3F7D3
:103E0000D7021207920793872703B3D7D702BD8B38
:103E1000D98FC207C1831EA445616FC0AFDA925724
:103E2000E1B791C55E250967D98F5EA582805A25C5
:103E3000F977FD17F98FD5BF13F7F50F8547158370
:103E4000B395B7006319F7009307C500984301CEF7
:103E5000D98D8CC38280894693074501E318D7FE2C
:103E600093070501E5B793C5F5FFF98DDDB70A2185
:103E70006D8D3335A000828013F7F50F85461583CD
:103E8000B397B6006311D7025A25F98F1A2101455D
:103E90004207418381CB0545A181B315B5006D8FE4
:103EA0003335E000828089466314D7001A29F1BFB8
:103EB0005A29E1BFA1818547B397B70093C7F7FFA0
:103EC000C207C1831EA1828001476314E600014539
:103ED0008280B307E5000507B386E5009C2383C60F
:103EE000F6FFE384D7FE3385D7408280B3C7A500B1
:103EF0008D8B3307C50081E78D4763EDC700AA8727
:103F0000637EE508942185078505A38FD7FEE3EB43
:103F1000E7FE828093763500AA8789CA94218507B7
:103F20008505A38FD7FE93F63700C5BF9376C7FFED
:103F3000138606FE63F0C70683A3050083A245002F
:103F400083AF850003AFC50083AE050103AE450115
:103F500003A3850183A8C5019385450223A07700AB
:103F600003A8C5FF23A2570023A4F70123A6E70156
:103F700023A8D70123AAC70123AC670023AE1701EA
:103F80009387470223AE07FF75B7904191079105CC
:103F900023AEC7FEE3EBD7FEE3E6E7F68280AA870F
:103FA00098239386170009EB850503C7F5FF85075E
:103FB000A38FE7FE75FB8280B687DDB7AA879821BD
:103FC00085078505A38FE7FE7DFB8280AA8785078D
:103FD00003C7F7FF6DFF3385A7407D15828015C2AB
:103FE0007D160147B307E500B386E5009C239422C4
:103FF0006396D7006304C7000507EDF73385D74004
:104000008280014582800000D04A0000E44A00001E
:10401000F44A0000084B0000144B0000204B000045
:10402000244B0000344B0000444B00004C4B00007C
:10403000604B0000704B0000784B0000844B000088
:10404000904B0000A44B0000AC4B0000BC4B0000A8
:10405000CC4B0000E44B00006D61696E0000000075
:10406000546F20696E697469616C697A6520646552
:10407000766963653A2573206661696C65642E20F4
:10408000546865206572726F7220636F6465206981
:10409000732025640A0000007469646C65000000E8
:1040A0000000010002000100030001000200010005
:1040B00004000100020001000300010002000100F1
:1040C00005000100020001000300010002000100E0
:1040D00004000100020001000300010002000100D1
:1040E00006000100020001000300010002000100BF
:1040F00004000100020001000300010002000100B1
:10410000050001000200010003000100020001009F
:104110000400010002000100030001000200010090
:10412000070001000200010003000100020001007D
:104130000400010002000100030001000200010070
:10414000050001000200010003000100020001005F
:104150000400010002000100030001000200010050
:10416000060001000200010003000100020001003E
:104170000400010002000100030001000200010030
:10418000050001000200010003000100020001001F
:104190000400010002000100030001000200010010
:1041A000303132333435363738394142434445466D
:1041B000000000000A205C207C202F0A0000000084
:1041C0002D205254202D202020202054687265611B
:1041D00064204F7065726174696E672053797374DF
:1041E000656D0A004D617920313220323032340061
:1041F000202F207C205C202020202025642E256478
:104200002E2564206275696C642025730A00000005
:104210002032303036202D203230313920436F703B
:104220007972696768742062792072742D7468727B
:10423000656164207465616D0A000000284E554C6C
:104240004C29000030313233343536373839616229
:104250006364656600000000746F74616C206D65B6
:104260006D6F72793A2025640A00000075736564E9
:10427000206D656D6F7279203A2025640A00000078
:104280006D6178696D756D20616C6C6F63617465CB
:1042900064206D656D6F72793A2025640A00000014
:1042A0006C697374206D656D6F72792075736167C9
:1042B0006520696E666F726D6174696F6E000000D3
:1042C0006C6973745F6D656D00000000746F20662B
:1042D000726565206120626164206461746120629E
:1042E0006C6F636B3A0A00006D656D3A203078257B
:1042F0003038782C207573656420666C61673A20CD
:1043000025642C206D6167696320636F64653A20C2
:104310003078253034780A0068656170000000004C
:104320006D656D20696E69742C206572726F7220E4
:10433000626567696E2061646472657373203078AA
:1043400025782C20616E6420656E6420616464723F
:1043500065737320307825780A0000001B5B324AB1
:104360001B5B48002D2D46756E6374696F6E204C83
:104370006973743A0A0000005F5F0000252D313632
:1043800073202D2D2025730A0000000064657669D6
:1043900063650000252D2A2E732020202020202058
:1043A0002020747970652020202020202020207279
:1043B000656620636F756E740A000000202D2D2D38
:1043C0002D2D2D2D2D2D2D2D2D2D2D2D2D2D2D2D1D
:1043D0002D202D2D2D2D2D2D2D2D2D2D0A000000C4
:1043E000252D2A2E2A7320252D32307320252D3895
:1043F000640A00006576656E74000000252D2A2E83
:1044000073202020202020736574202020207375C5
:104410007370656E64207468726561640A000000E0
:1044200020202D2D2D2D2D2D2D2D2D2D202D2D2DE3
:104430002D2D2D2D2D2D2D2D2D2D2D0A0000000083
:10444000252D2A2E2A7320203078253038782025F3
:104450003033643A00000000252D2A2E2A732020D4
:1044600030782530387820300A0000006D61696CA2
:10447000626F7800252D2A2E7320656E7472792064
:1044800073697A652073757370656E6420746872E1
:104490006561640A00000000202D2D2D2D20202DA7
:1044A0002D2D2D202D2D2D2D2D2D2D2D2D2D2D2D49
:1044B0002D2D0A00252D2A2E2A7320253034642024
:1044C00020253034642025643A000000252D2A2E52
:1044D0002A7320253034642020253034642025645C
:1044E0000A0000006D736771756575650000000056
:1044F000252D2A2E7320656E747279207375737062
:10450000656E64207468726561640A00202D2D2D2B
:104510002D20202D2D2D2D2D2D2D2D2D2D2D2D2DE5
:104520002D0A0000252D2A2E2A73202530346420E0
:104530002025643A00000000252D2A2E2A7320250C
:10454000303464202025640A000000006D75746515
:1045500078000000252D2A2E732020206F776E65AD
:10456000722020686F6C642073757370656E6420B0
:104570007468726561640A00202D2D2D2D2D2D2D5E
:104580002D202D2D2D2D202D2D2D2D2D2D2D2D2D75
:104590002D2D2D2D2D0A0000252D2A2E2A732025A4
:1045A0002D382E2A7320253034642025640A00001B
:1045B00073656D6170686F7265000000252D2A2E8D
:1045C00073207620202073757370656E6420746884
:1045D000726561640A000000202D2D2D202D2D2DE7
:1045E0002D2D2D2D2D2D2D2D2D2D2D0A00000000D2
:1045F000252D2A2E2A7320253033642025643A0085
:10460000252D2A2E2A7320253033642025640A00A4
:104610007468726561640000252D2A2E7320707203
:10462000692020737461747573202020202020730A
:10463000702020202020737461636B2073697A6579
:10464000206D61782075736564206C6566742074D4
:1046500069636B20206572726F720A00202D2D2D08
:1046600020202D2D2D2D2D2D2D202D2D2D2D2D2DA1
:104670002D2D2D2D202D2D2D2D2D2D2D2D2D2D2084
:10468000202D2D2D2D2D2D20202D2D2D2D2D2D2D81
:104690002D2D2D202D2D2D0A00000000252D2A2E38
:1046A0002A732025336420002072656164792020FC
:1046B000000000002073757370656E6400000000D8
:1046C00020696E69742020200000000020636C6F58
:1046D00073652020000000002030782530387820D5
:1046E0003078253038782020202025303264252568
:1046F00020202030782530387820253033640A0097
:1047000074696D6572000000252D2A2E73202070BB
:104710006572696F64696320202074696D656F75C7
:104720007420202020202020666C61670A00000091
:10473000202D2D2D2D2D2D2D2D2D2D202D2D2D2DC3
:104740002D2D2D2D2D2D202D2D2D2D2D2D2D2D2DA6
:104750002D2D0A00252D2A2E2A7320307825303859
:104760007820307825303878200000006163746943
:1047700076617465640A00006465616374697661DA
:104780007465640A0000000063757272656E7420BF
:104790007469636B3A3078253038780A000000007D
:1047A0006C69737420616C6C2073796D626F6C201E
:1047B000696E2073797374656D0000006C697374A1
:1047C000000000006C69737420646576696365207D
:1047D000696E2073797374656D0000005F5F636DAF
:1047E000645F6C6973745F6465766963650000007B
:1047F0006C6973742064657669636520696E2073E3
:10480000797374656D0000006C6973745F6465761C
:10481000696365006C6973742074696D65722069E1
:104820006E2073797374656D000000005F5F636DC7
:10483000645F6C6973745F74696D65720000000079
:104840006C6973742074696D657220696E20737968
:104850007374656D000000006C6973745F74696D3A
:10486000657200006C697374206D657373616765B0
:1048700020717565756520696E2073797374656D37
:10488000000000005F5F636D645F6C6973745F6D4F
:1048900073677175657565006C697374206D6573F8
:1048A0007361676520717565756520696E20737920
:1048B0007374656D000000006C6973745F6D7367DD
:1048C00071756575650000006C697374206D6169B0
:1048D0006C20626F7820696E2073797374656D0047
:1048E0005F5F636D645F6C6973745F6D61696C6257
:1048F0006F7800006C697374206D61696C20626F61
:104900007820696E2073797374656D006C697374B7
:104910005F6D61696C626F78000000006C69737490
:10492000206D7574657820696E2073797374656D78
:10493000000000005F5F636D645F6C6973745F6D9E
:1049400075746578000000006C697374206D75746F
:10495000657820696E2073797374656D00000000BE
:104960006C6973745F6D7574657800006C6973743D
:10497000206576656E7420696E2073797374656D39
:10498000000000005F5F636D645F6C6973745F6556
:1049900076656E74000000006C697374206576653E
:1049A0006E7420696E2073797374656D0000000069
:1049B0006C6973745F6576656E7400006C697374FE
:1049C0002073656D6170686F726520696E20737900
:1049D0007374656D000000005F5F636D645F6C69F8
:1049E00073745F73656D00006C6973742073656D1B
:1049F0006170686F6E6520696E2073797374656D80
:104A0000000000006C6973745F73656D0000000046
:104A10006C69737420746872656164005F5F636DB4
:104A2000645F6C6973745F74687265616400000030
:104A30006C69737420746872656164006C69737466
:104A40005F74687265616400746865207465726D76
:104A5000696E616C2073637265656E005F5F636D84
:104A6000645F636C65617200746865207465726D63
:104A7000696E616C2073637265656E00636C65615D
:104A8000720000007265626F6F7420746865206246
:104A90006F617264000000005F5F636D645F726548
:104AA000626F6F74000000007265626F6F74207433
:104AB000686520626F617264000000007265626F59
:104AC0006F7400002D000000257300002F0000000F
:104AD00043686172616374657220446576696365D9
:104AE00000000000426C6F636B204465766963656B
:104AF000000000004E6574776F726B20496E74651C
:104B000072666163650000004D5444204465766917
:104B10006365000043414E2044657669636500008B
:104B200052544300536F756E642044657669636523
:104B3000000000004772617068696320446576690F
:104B4000636500004932432042757300555342208B
:104B5000536C6176652044657669636500000000EA
:104B600055534220486F7374204275730000000053
:104B7000535049204275730053504920446576696B
:104B8000636500005344494F2042757300000000E4
:104B9000504D2050736575646F2044657669636578
:104BA000000000005069706500000000506F7274D2
:104BB000616C2044657669636500000054696D6529
:104BC0007220446576696365000000004D69736377
:104BD000656C6C616E656F7573204465766963659D
:104BE00000000000556E6B6E6F776E00546F6F2083
:104BF0006D616E7920617267732021205765206F87
:104C00006E6C79205573653A0A0000002573200008
:104C100025733A20636F6D6D616E64206E6F742032
:104C2000666F756E642E0A0052542D546872656169
:104C300064207368656C6C20636F6D6D616E647366
:104C40003A0A00005F5F636D645F0000252D313616
:104C500073202D2025730A0052542D54687265610B
:104C600064207368656C6C2068656C7000000000DF
:104C70005F5F636D645F68656C70000053686F7799
:104C800020746865206D656D6F727920757361673A
:104C90006520696E207468652073797374656D0092
:104CA0005F5F636D645F6672656500004C69737475
:104CB000207468726561647320696E207468652071
:104CC00073797374656D00005F5F636D645F70730B
:104CD000000000006D7368200000000066696E73BC
:104CE000682000003E00000066696E73683A206329
:104CF000616E206E6F742066696E642064657669EB
:104D000063653A2025730A006E6F206D656D6F72C2
:104D10007920666F72207368656C6C0A0000000071
:104D2000747368656C6C0000736872780000000032
:104D300008000000256300000825732020080000FB
:104D4000082008001B5B324B0D0000002573257303
:104D500000000000726561642073746174757320D3
:104D600066726F6D20686172647761726520706928
:104D70006E00000070696E5265616400777269743C
:104D8000652076616C756520746F20686172647748
:104D90006172652070696E0070696E577269746522
:104DA0000000000073657420686172647761726549
:104DB0002070696E206D6F646500000070696E4D33
:104DC0006F64650075617274310000001830000076
:104DD000D82F0000FA2F0000963000002831000084
:104DE00082310000010000001600000002000000F7
:104DF0001700000004000000180000000800000078
:104E000019000000100000001A000000200000003F
:104E10002700000040000000270000008000000084
:104E20002700000000010000270000000002000031
:104E30002700000000040000380000000008000007
:104E400038000000001000003800000000200000C2
:104E50003800000000400000380000000080000022
:104E600038000000FFFFFFFF00000000000000000E
:104E700000000000010000008A2F0000001801401F
:104E800004000000020000008A2F0000001801400A
:104E900008000000030000008A2F000000180140F5
:104EA00010000000040000008A2F000000180140DC
:104EB00020000000050000008A2F000000180140BB
:104EC00040000000FFFFFFFF0000000000000000A6
:104ED00000000000070000007A2F000000100140D1
:104EE00000200000080000007A2F000000100140A0
:104EF00000400000090000007A2F0000001001406F
:104F000000800000FFFFFFFF000000000000000025
:104F100000000000FFFFFFFF000000000000000095
:104F200000000000FFFFFFFF000000000000000085
:104F300000000000FFFFFFFF000000000000000075
:104F400000000000FFFFFFFF000000000000000065
:104F5000000000000F0000007A2F00000010014048
:104F600001000000100000007A2F00000010014036
:104F700002000000110000007A2F00000010014024
:104F800004000000120000007A2F00000010014011
:104F900008000000FFFFFFFF00000000000000000D
:104FA00000000000FFFFFFFF000000000000000005
:104FB00000000000FFFFFFFF0000000000000000F5
:104FC00000000000FFFFFFFF0000000000000000E5
:104FD00000000000170000006A2F000000080140D8
:104FE00001000000180000006A2F000000080140C6
:104FF00002000000190000006A2F000000080140B4
:10500000040000001A0000006A2F000000080140A0
:1050100008000000FFFFFFFF00000000000000008C
:1050200000000000FFFFFFFF000000000000000084
:10503000000000001D0000006A2F00000008014071
:10504000100000001E0000006A2F00000008014050
:10505000200000001F0000006A2F0000000801402F
:1050600040000000200000006A2F000000080140FE
:1050700080000000210000007A2F00000010014095
:1050800010000000220000007A2F000000100140F4
:1050900020000000230000005A2F0000000C0140F7
:1050A00001000000240000005A2F0000000C014005
:1050B00002000000250000005A2F0000000C0140F3
:1050C00004000000260000008A2F000000180140A4
:1050D00080000000270000008A2F00000018014017
:1050E00000010000280000008A2F00000018014085
:1050F00000020000290000008A2F00000018014073
:10510000000400002A0000008A2F0000001801405F
:10511000000800002B0000008A2F0000001801404A
:10512000001000002C0000008A2F00000018014031
:10513000002000002D0000008A2F00000018014010
:10514000004000002E0000008A2F000000180140DF
:10515000008000002F0000005A2F0000000C0140CA
:1051600000040000300000005A2F0000000C014035
:1051700000080000FFFFFFFF00000000000000002B
:1051800000000000FFFFFFFF000000000000000023
:1051900000000000330000005A2F0000000C014006
:1051A00000100000340000005A2F0000000C0140E5
:1051B00000200000350000005A2F0000000C0140C4
:1051C00000400000360000005A2F0000000C014093
:1051D0000080000037000000482F0000001401404C
:1051E0000001000038000000482F000000140140BA
:1051F0000002000039000000482F000000140140A8
:10520000000400003A000000482F00000014014094
:10521000000800003B000000482F0000001401407F
:10522000001000003C000000482F00000014014066
:10523000002000003D000000482F00000014014045
:10524000004000003E000000482F00000014014014
:10525000008000003F0000007A2F00000010014095
:1052600040000000400000007A2F000000100140C4
:1052700080000000410000007A2F00000010014073
:1052800000010000420000007A2F000000100140E1
:1052900000020000430000006A2F000000080140E7
:1052A00000010000440000006A2F000000080140D7
:1052B00000020000450000006A2F000000080140C5
:1052C00000040000460000006A2F000000080140B2
:1052D00000080000470000006A2F0000000801409D
:1052E00000100000480000006A2F00000008014084
:1052F00000200000FFFFFFFF000000000000000092
:1053000000000000FFFFFFFF0000000000000000A1
:1053100000000000FFFFFFFF000000000000000091
:10532000000000004C0000006A2F0000000801404F
:10533000004000004D0000006A2F000000080140FE
:10534000008000004E0000007A2F00000010014095
:10535000000400004F0000007A2F00000010014000
:1053600000080000500000007A2F000000100140EB
:105370000010000051000000482F00000014014000
:105380000100000052000000482F000000140140FE
:105390000200000053000000482F000000140140EC
:1053A0000400000054000000482F000000140140D9
:1053B0000800000055000000482F000000140140C4
:1053C0001000000056000000482F000000140140AB
:1053D0002000000057000000482F0000001401408A
:1053E0004000000058000000482F00000014014059
:1053F00080000000590000005A2F0000000C0140FE
:10540000080000005A0000005A2F0000000C014064
:10541000100000005B0000005A2F0000000C01404B
:10542000200000005C0000005A2F0000000C01402A
:10543000400000005D0000005A2F0000000C0140F9
:1054400080000000FFFFFFFF0000000000000000E0
:10545000000000005F0000005A2F0000000C014017
:1054600000010000600000005A2F0000000C014005
:1054700000020000610000008A2F000000180140B7
:1054800001000000620000008A2F000000180140A7
:1054900002000000FFFFFFFF00000000000000000E
:1054A00000000000FFFFFFFF000000000000000000
:1054B0000000000070696E00B23400008036000009
:1054C0005E3600003C360000AE3400002068617299
:1054D0006466756C740D0A00204E4D492048616E5B
:1054E000646C65720D0A00000D0A204D43553A2088
:1054F00043483332563330330D0A0000205379735A
:10550000436C6B3A202564487A0D0A002043686991
:105510007049443A20253038780D0A002077777793
:105520002E7763682E636E0D0A000000C0420000F3
:10553000A0420000D0100000BC470000A0470000BF
:105540006C210000DC470000C44700003E20000042
:1055500008480000F04700003E2000002C480000F2
:1055600014480000D22000005848000040480000C5
:10557000D22000008448000064480000881F00001A
:10558000B848000098480000881F0000E04800006C
:10559000C8480000CA1E00000C490000F448000082
:1055A000CA1E0000344900001C490000481E0000CB
:1055B0006049000048490000481E0000844900007E
:1055C0006C4900009C1D0000B04900009849000093
:1055D0009C1D0000D8490000BC490000E61C0000EA
:1055E000044A0000E8490000E61C00001C4A0000D4
:1055F000104A0000061C00003C4A0000304A00002F
:10560000061C00005C4A0000484A00005C1B0000C9
:105610007C4A0000684A00005C1B0000984A0000B9
:10562000844A00004A1B0000BC4A0000A84A00004F
:105630004A1B0000704C0000584C0000B6210000CE
:10564000A04C00007C4C00006C240000C84C000002
:10565000AC4C00005E240000744D0000544D00006E
:10566000BC2D0000984D00007C4D0000A22D0000D4
:10567000BC4D0000A44D0000882D0000A6040000D1
:10568000AE0400009C2F00007C350000B204000036
:085690008C240000AA040000B4
:105698000100000004000020040000208000000039
:1056A8000200000014000020140000202000000068
:1056B8000300000024000020240000202400000033
:1056C8000400000034000020340000202000000006
:1056D80005000000440000204400002030000000C5
:1056E8000600000054000020540000203400000090
:1056F800090000006400002064000020440000004D
:105708000A00000074000020740000202C00000033
:10571800FFFF00000000000000000000FFFF000085
:105728000000000000000000FFFF00000000000073
:1057380000000000FFFF0000000000000000000063
:10574800FFFF00000000000000000000FFFF000055
:105758000000000000000000FFFF00000000000043
:1057680000000000FFFF0000000000000000000033
:10577800FFFF00000000000000000000FFFF000025
:105788000000000000000000FFFF00000000000013
:1057980000000000FFFF0000000000000000000003
:1057A800FFFF00000000000000000000FFFF0000F5
:1057B8000000000000000000FFFF000000000000E3
:1057C80000000000FFFF00000000000000000000D3
:1057D8000000000000000000010203040607080999
:1057E800000000000102030401020304060708097F
:0857F80000D8B8050204060800
:00000001FF
